:020000020000FC
:040000000C948200DA
:1001000000EC05BFC0EDD0E000E003500DBF01E002
:1001100000400EBF0E944701002309F424D0E0E60E
:10012000F0E000E110E00E944217E0E0F0E000E0C3
:1001300010E040E050E00E943417E4E0F1E00CE50C
:1001400013E00E944217EEE3F2E000E011E044E029
:1001500050E00E943417EAE6F1E000E614E040E0E7
:0A01600050E00E9434170C9449018E
:04028E0001E00895EE
:100292000E944A07002319F40E947403FDCFF894C8
:0C02A2000E94840178940E94A301FDCF0B
:10016A000A53494F32494445207665722E20332E70
:10017A00302028632932303032204D4D536F667457
:02018A000A0069
:1002AE005798E2E6FF2700831183E0E6F083F1839F
:1002BE00E4E6F083579A089519B71D7F19BF00938E
:1002CE00060209B7026009BF089509B70D7F09BF7D
:1002DE0000910602002311F0002701C001E019B7BA
:1002EE00126019BF08950EEFE7DF04E010E0D8DFCB
:1002FE00949A01E00093040208958C9A909A07E173
:10030E0009B908E90AB98A98929A07EB02BF05E083
:10031E0003BF09B7026009BFE6CF000F111F202FE0
:10032E00312F01501040232B11F00000F8CF08950B
:10033E005D9BFECF0CB908950E945617A4E0B1E064
:10034E00C4DF002309F0CFDF00910402E2E4F2E003
:10035E000C94D716829BA6C00EEFAEDFEA2FFB2FB2
:10036E0041810A2F1B2F0E946A07002309F499C0AE
:10037E00002700930502B0D0E457FE4FC895002029
:10038E0009F48DC0A9D0E457FE4FC895EA2FFB2F74
:10039E000181001621F5A0D0AAD0002901F1552720
:1003AE0000910502112746E00E943816E02FF12F2A
:1003BE009ED0E02FF02D42E650E00A2F1B2F09951C
:1003CE00002369F089D0E157FE4FC89500920402D0
:1003DE00E2E6FF270081118163DF949863C00091EC
:1003EE0005020395C6CF08EC10E06BD009F44EC0A1
:1003FE0073D0E057FE4FC89570D009F447C003E4A0
:10040E0097DF07E036C042C041C00AEF10E085DF3B
:10041E004ED030F5E0E6008111810C5F1E4FE02FCB
:10042E00F12F008185DFFF2704E610E0E0E6208152
:10043E00318166D03327E4E6FF274081240F331F36
:10044E003150E0E62081318118F05AD0239501C059
:10045E0057D0E02FF12F0081020F008357D0D8CF55
:10046E00E4E600811DC04AD002E026DF01E460DF31
:10047E0004E00093040216C000ED17E022D031F024
:10048E002BD0E057FE4FC89528D021F405E408C0C4
:10049E0035D04ED003E404C004EF11E03EDF0EE48D
:1004AE0047DF21DFE4E00C94671702E005DFE0E6AA
:1004BE00FF2700811181E2E62081318102171307A7
:1004CE0008952BDF35D02AD0E057FE4FC895002D6A
:1004DE003196C8950029089521C0002D3196C895F2
:1004EE00E02FF02D04E011E0099500230895E35765
:1004FE00FE4FC895002D3196C895089508EC1BC087
:10050E002C5F3E4FE22FF32F20810895E0E600810D
:10051E0011810F5F1F4F0083118308950091050213
:10052E00112746E050E00E943816E02FF12F089573
:10053E0001E4FEDE0AEF10E0F0CE0A921A922A9241
:10054E003A920A931A932A933A934A935A936A9336
:10055E007A93EA93FA93FFB7FA938A938CB18299BE
:10056E0019C0009104020130A9F49FDF50F441D06C
:10057E00082F08F00395E22FF32F1081100F108330
:10058E0009C0E4E60081081711F402E001C008E09A
:10059E0000930402829B1BC0009104020430B9F444
:1005AE0084DF48F426D008F08395E22FF32F0081E4
:1005BE00080F00830CC00EEF7FDEE4E6FF270081FC
:1005CE00081711F405E001C009E0009304028991B7
:1005DE00F991FFBFF991E9917991699159914991F9
:1005EE003991299119910991399029901990099071
:1005FE0018958CDF015010400C5F1E4FE02FF12F2D
:10060E008083E4E6FF2724E630E0082F112740819F
:10061E00040F1F1F115008950A93EA93FA93FFB720
:10062E00FA93009106020E3F49F000910602002354
:10063E0029F00091060201500093060207EB02BF5B
:0C064E00F991FFBFF991E991099118950D
:10024200020059020900B1013A0259024302FA01BD
:080252000C02580253024F0296
:04002C000C9413031A
:040034000C94A40282
:10065A00000F111F221F331F35D0015010402040B8
:10066A003040452B462B472B11F00000F5CF08955B
:10067A002ED00E949A16742E7394082F192F2A2F9F
:10068A003B2FE42D24D00E949A16E42D23D00E94F9
:10069A009A16642E2A2F3B2FE42D0381148142815E
:1006AA0055270E943816402F512F66277727082F83
:1006BA00192F0E949A16402E512E062D0F700056A1
:1006CA00602E0895402F512F622F732F0895438172
:1006DA00548102C04281552766277727089500EA88
:1006EA0016E821E030E0B4DFAD9800E41DE023E035
:1006FA0030E0AEDFAD9A089531E040E811273323A8
:10070A0039F0202F232309F0142B330F4695F7CF06
:10071A00012F08959A938A93902F042F852FECDF47
:10072A001FEF1ABB17BBF89415B3107E192B15BB14
:10073A00AF980BBB88BBAF9A000005B30F6105BB2E
:10074A0078940FEF0ABB0BBB07BB08BB8991999141
:10075A0008959A938A9311271ABB1FEF1BBB11277F
:10076A0017BB1FEF18BBF89415B3107E102B15BBDF
:10077A00AE980000AE9A09B386B315B31F6115BBD4
:10078A0078941FEF1ABB1BBB17BB18BBB5DF182F1A
:10079A008991999108950E945717A02F80E197E2B5
:1007AA00AA2339F00197082F092B19F4AD980027CD
:1007BA0005C00DE1CEDF00309CF301E0E3E00C94CC
:1007CA00681711D0882339F011970A2F0B2B19F4C7
:1007DA00AD98002705C00DE1BCDF06FFF3CF01E0AD
:1007EA00E4E00C9467170E945617802FA0E1B7E245
:1007FA000895F9DF882339F011970A2F0B2B19F482
:10080A00AD98002705C00DE1A4DF03FFF3CF01E097
:10081A00E4E00C9467170DE19CDF00FF03C0AD987C
:10082A0001E00895AD9A0027089522D0B0F0E42D92
:10083A00F52D01850030042F2CF0152F262F372F88
:10084A0017DF01C025D011D041F02BD041E209D0E9
:10085A0021F03BD011F401E001C00027E8E00C943C
:10086A00631750E00DE156DF33C005E072DF34C094
:10087A000E945217402E512E842F952FA62FB72F44
:10088A00E02FF12F2DD004171507260737070895F3
:10089A00702E492E5A2E6B2E0FE0602200EE600E4B
:1008AA000895462D552709E135DF41E050E009E07A
:1008BA0031DF472D55270DE02DDF442D552701E166
:1008CA0029DF452D50E005E125CFA5DF0023089556
:1008DA0001E08FDF0023089501E05DDF0023089522
:1008EA0005811681278130850895C2DFB8F0E42D8D
:1008FA00F52D018506FD12C0E42DF52D0185003088
:10090A00082F2CF0192F2A2F3B2FB2DE01C0C0DF8F
:10091A00ACDF21F0C6DF41E3A4DF11F4002701C0F8
:10092A0001E0E8E00C946317082F192F2A2F3B2FB8
:10093A0042E00C9491160E945617802F912F2AD0CC
:10094A00A0E0B1E0E02FF12F218526FF0EC022277B
:10095A0033273A932A937A936A935A934A93402F66
:10096A00512F082F192F4FD112C05FDF002371F0CA
:10097A000A2F1B2F1197012B01E049F0EADEE82F1D
:10098A00F92F019311938E2F9F2FF2CF0027E8E0C2
:10099A000C946717042F152F4C815D816E817F811E
:1009AA0008950E945617A02FB12FF4DF80E091E03E
:1009BA00E02FF12F218526FD12C097DF002379F061
:1009CA00082F192F0197012B21F04D915D910ED01F
:1009DA00F7CF82DF21F079DF11F401E001C00027AF
:1009EA00E8E00C946717A02FB12F3FCF01E092CE19
:1009FA000E945417F8DF09F46AC071D04CEE31DF57
:100A0A0009F465C062DF09F062C04424552401E09C
:100A1A00501608F042C05FD0042D152DEAE5F2E029
:100A2A000C94DB1600E09030A4F552C0EA2FFB2F9D
:100A3A00808391832EC0EA2FFB2F82832AC0EA2F5C
:100A4A00FB2F8383948325C091FF23C0EA2FFB2FBA
:100A5A000185006801871DC0EA2FFB2F0185003040
:100A6A00C4F42227858396832783208712C0EA2F1E
:100A7A00FB2F018500306CF411274581568167816F
:100A8A007085410F511F681F791F458356836783FD
:100A9A0070870FEF401A500ABACFEA2FFB2F018551
:100AAA0000309CF0008111812227332713DE0E9437
:100ABA006C16EA2F0CDE0E946C16EA2F14D010DF97
:100ACA0001501040204030400ED001E001C0002704
:100ADA00E6E00C9465173DDE802F912F089540EAD9
:100AEA0050E009E117CE05831683278330870895DE
:100AFA00BCDE11F400270895F2DF4CE050E001E17A
:100B0A001BD005E119D005E017D009E015D00DE09A
:100B1A0013D001E1FFDD48E050E005E1FBDD40EAEA
:100B2A00A0DE11F400270895D7DE11F400270895F6
:100B3A0001E0089550E001E0EDDD442755270895CE
:100B4A000E944C17A02EB12E442E552E662E772EBB
:100B5A0088889988AE85BF85CC2404E0D02EC8DF6A
:100B6A00002309F44CC048EA50E040DF472D562DD7
:100B7A003DDF452D542DDFDF39DF40E051E0DBDF7B
:100B8A0035DF002708DE0023D1F1002732DE0023FB
:100B9A00B1F19BDEA1F52C2D3D2D0FEFC00ED01E1D
:100BAA00232B01E011F197DF0A2F0B2B11F011977C
:100BBA000BC0082D092941F00FEF800E901EEA2D77
:100BCA00FB2D8193AE2EBF2E0A2F0B2B11F01197FE
:100BDA00E2CF082D0929F9F20FEF800E901EEA2DB7
:100BEA00FB2D9193AE2EBF2ED6CF03DE002329F024
:100BFA0001E0AFDD6DDEE1F702C001E001C00027D0
:100C0A00E2E10C945D170E945217602E712E4C84FB
:100C1A005D8488859985AA85BB85E42FF52F018592
:100C2A0006FF58C05DDE80179107A207B30708F0D8
:100C3A0051C001E0401602E0500608F04BC0042DF6
:100C4A000529B9F1082F037011272227332703300A
:100C5A0010402040304069F567DE802F912FA22F87
:100C6A00B32F00E012E0041915091A930A93042D10
:100C7A00152D1A5F1A930A93482F592F622F732F33
:100C8A002FD009F427C08F5F9F4FAF4FBF4F5A92A3
:100C9A004A92002711271A930A93482F592F6A2F2D
:100CAA007B2F64187508600E02E0701E19D0A1F43B
:100CBA0011C000E012E01A930A93082F0370102F54
:100CCA000027110F040D151D1A930A932DDEFADC65
:100CDA0007D011F4002701C001E0EEE00C9463177D
:100CEA00062D172D2DDF002308950E9456177BDE4F
:100CFA0069F1F5DE41EAB5DD49F1E7DD39F5882725
:100D0A00992701E09130B0F424DD282F392F2050A3
:100D1A00304021F02153304021F00AC0103044F015
:100D2A0015C011FF13C0EA2FFB2F01850068018748
:100D3A000196E7CFEA2FFB2F01850064018700E8BF
:100D4A0011E327E130E0CFDE01E001C00027E4E053
:100D5A000C9467170E945217402E512E642E752E3E
:100D6A00C7DE002319F143E0E5DE40DE42E1E2DEC0
:100D7A00E2DEE1DE3BDEB0DDC9F0AADDB9F0A5DDD9
:100D8A00A9F4AA27BB27EA2FFB2F399701E078F4A9
:100D9A00A2DE0A2F1B2F0650104031F4E42DF52D48
:100DAA008083E62DF72D90831196EDCF0027E8E09A
:100DBA000C9463172297E02FF12F018506FF0EC0CE
:100DCA004C2F5D2F4F5F5F4F0C2F1D2FC3DF00236A
:100DDA0039F00881E4E7F2E00C94D71601E001C08B
:100DEA000027229608959A938A93802F912F00279D
:100DFA00E82FF12F00830183028303830483058391
:100E0A000683078300870187082F6FDF002339F0E5
:100E1A00082F192FCFDF0023D9F302E008C0082FCB
:100E2A00192FE6DD002311F001E001C000278991A6
:100E3A009991089554DE4EE050E00AE16BDC0AE035
:100E4A0010E020E030E004DC4AE050E00AE162DC35
:100E5A0000E211EA27E030E0FBDB00279CCC9A9302
:100E6A008A93802F912F0FEF0ABB0BBB07BB08BBDE
:100E7A0004BB0FE105BBAE9AAF9AAD98DBDF082F32
:0A0E8A00192FB1DF899199910895A5
:10025A000000014E051705011B05022005032405B0
:10026A002B29050B3105013C05FB0001F506F306B8
:10027A0002F50602F50624F50601F50611F506C58E
:03028A00F506FB7B
:100E94008D988E988F98959A969A979A00B3003069
:100EA4008B9A14F0939801C0939AE5E6FF27F08398
:100EB4000E94DB14002311F40027089500B30030CE
:100EC4000CF08B9A939A01E0E5E6FF2700830895DE
:100ED400E02FF12F2081213711F4859B07C0E02FEB
:100EE400F12F2081223701F5859B1EC04131C1F0CD
:100EF4004231B1F04631A1F0433191F0443181F0F7
:100F0400453171F0473161F0483151F0493141F0D8
:100F14004A3131F04B3121F04C3111F04D3111F4A3
:100F240001E0089500270895E02FF12F2081213357
:100F340018F02081293310F00027089520B32030C1
:100F44003CF4E02FF12F2081213311F40027089580
:100F540086990EC0E02FF12F2081213311F422E372
:100F640006C0E02FF12F2081223311F421E32083E6
:100F7400E02FF12F008100530E942E12012B11F05B
:100F840001E0089500270895E02FF12F20812053D8
:100F9400209307022381028100930802209309020F
:100FA400009107020E942E1220910802309109023A
:100FB4000217130708950CD00CE010E0E42FF52F6E
:100FC40000831183009107020E942E12012B0895C1
:100FD400E02FF12F008100530093070208951DD0E4
:100FE40031F0D2DF20F0022F132F032B11F400274E
:100FF40011C0E22FF12F319738F0E22FF12F3497FF
:1010040018F400E810E001C015D0E82FF92F008390
:10101400118301E08991999108959A938A93842F79
:10102400952FE5E6FF272081222308959A938A933A
:10103400802F912F009107020C941C1202D00C9463
:10104400B8131A930A93409108025091090200912F
:1010540007020895E2DF31F097DF20F0022F132F0B
:10106400032B11F4002711C0E22FF12F319738F030
:10107400E22FF12F349718F400E810E001C0DADF12
:10108400E82FF92F0083118301E089919991089544
:10109400D8DF0C943A139CDF04E00FD00AD0012B64
:1010A40011F400270895E5E6FF27008108958E2FA7
:1010B4009F2F009107020C942E1210E0E42FF52FBD
:1010C400008311830895B2DF0030114011F400E36E
:1010D40001C000E1E82FF92F01930FEF019300EE17
:1010E40001930027008301E089919991089563DFBA
:1010F400D1F600270895D7CF9A938A93802F01E0E1
:10110400E82FF12F019300E10193D1DFE82FF92FAC
:101114001193CDDFE82FF92F0193002701938E2F30
:101124009F2F88DF0030114041F40CE0E82FF92FA5
:10113400019301E00193002707C008E0E82FF92F8D
:1011440001930027019300E8019300E4019309E46B
:10115400019304E4019305E4C5CF2DDF09F0A3CF87
:1011640000270895A0CF9A938A93E02FF12F8281CC
:10117400982F0381802F9DDF0817190711F000278E
:1011840001C001E08991999108959A938A93842FDB
:10119400952F1EDF0E941C12E82FF92F0083118364
:1011A40000811181012B11F4002703C0E5E6FF271C
:1011B400008189919991089539DF025010402FEFF1
:1011C400E82FF92F21932193202F312F0150104024
:1011D400232B09F488CF2227F6CF85CF1A930A93BD
:1011E4000027E42FF52F00830183229608951A9394
:1011F4000A93002722960895E02FF12F028100938D
:1012040007020FE05ADF009107020C941412402FDA
:10121400512F009107020C943811EECF402F512F1B
:10122400009107020C9463111A930A930FE045DFAF
:10123400E5E6FF270081229608950C940811F4CF67
:101244000C94241121E030E0E42FF52F2083318326
:10125400E02FF12F02810C94F6112FEFE02FF12FE4
:10126400208321CF1A930A9301E0E1CF2FEFE02FDF
:10127400F12F20830C9442121A930A930AE0D7CFD9
:101284000E94B21201E008951A930A9304E0CFCFAA
:101294000E94B81201E008951A930A930FE0C7CF91
:1012A4000C94AF10F9CF0C94C310F6CF0C94D31058
:1012B400F3CF0E94E01001E00895EECF9A938A9351
:1012C400802F912F0E944214002339F0082F192FE8
:1012D4000E94E0100E94041106CF0FE010E01A9360
:1012E4000A9344275527082F192F0E94AD17FBCEC8
:10018C00534D0806650850F10703200857F1070383
:10019C002008522C08064A084E7908067E084FAFF4
:1001AC000803B50821C70806DE083FF00806F90861
:1001BC0011FE08060909120F090310091316090686
:1001CC001F091421090622091634090638091524B9
:1001DC0009062F09173E09064209184609064A095D
:1001EC00194E090652091A54090655091B570903D9
:1001FC0058091C5A09065B091D5F090660090000B5
:04020C0000010000ED
:1012F4000E945617802F912FA22FB32FE0E0F1E028
:1013040061D069D089F0BA93AA939A938A936CD0E6
:101314000E94A004002311F4002707C0E0E0F1E0DC
:1013240080839183A283B38301E0E4E00C94671784
:101334000E945617802F912FA42FB52F5AC0222711
:10134400332701505CD05FD0802F912FA22FB32F71
:10135400082D5FD0E65FFB4F00811181228133812C
:10136400800F911FA21FB31F0895041B150B260B9A
:10137400370B409154045527662777270E949A1605
:10138400802F912FA22FB32F8E5F9F4FAF4FBF4F50
:101394000895802F912FA22FB32F823000E01007E1
:1013A400200730070895802F912FA22FB32F0F3FCE
:1013B4001F4F08950E945217602E712E442E552EF1
:1013C400E5E5F4E0008111812281338108958F5F86
:1013D4009F4FAF4FBF4F80179107A207B3070895E0
:1013E4003A932A931A930A9346E655270AE012E0A1
:1013F400089542EB5DE099D2002308950250104015
:10140400204030400895442D552D662777270C94AD
:101414009A16112747E050E00E943816E02FF12F6A
:1014240008955A934A93DCDF0C940806D9DF0C9490
:10143400D6040E945617802F012F122F232F3327F3
:1014440031D019F40027112705C0E82FFF2734D025
:101454000081118122273327E4E00C946717082FB9
:10146400CDDF409154045527662777270E946C16D8
:1014740035D03BC0E2E4F4E03DC0E2E4F4E00584AE
:1014840016842784308881859285A385B4850816BF
:1014940019062A063B06089521D040175107620712
:1014A40073070895E2E4F4E0418152816381748119
:1014B4001CD01EDF00230895EE0FFF1FE65FFD4FD3
:1014C4000895E2E4F4E00584168427843088E5E591
:1014D400F4E000821182228233820895E2E4F4E08F
:1014E40045815681678170850895040F151F261F55
:1014F400371F0895018512852385348508950E9438
:101504005617802F47E00E949116CCDF29F400275C
:1015140011272227332708C0E82FEF77FF27EE0F84
:10152400FF1FCADF4FDF3F70E4E00C9467170E948F
:101534005217602E712EE02FF12F44DFADDF28F417
:10154400E62DF72D3FDF11DF01C050D04424552490
:1015540000914204045039F0025029F00650E9F099
:101564000357B9F139C0082F192F2A2F3B2F61DFF8
:10157400402F412B422B432B79F14FEF441A540A4D
:101584000F3F140740E02407340711F020DF21F552
:101594000ADF2040304039F719C0082F192F2A2FAD
:1015A4003B2FADDF402F412B422B432BA9F04FEFB4
:1015B400441A540A0F3F140724074FE0340711F06C
:1015C40006DF51F4F0DE2F4F3F4039F7042D152D7F
:1015D4000AC001E010E007C0E62DF72D0681006285
:1015E400068300271127E8E00C94631782E090E05B
:1015F400A0E0B0E008950CD0065F1F4F0E94DB15F9
:101604000051FDDE442D552D662777270C949A163C
:1016140000915B0410915C0408950E945617802F7A
:10162400912FA42FB52FCCDE5BDF3CD090F5009139
:101634005904112745E00E944816065F1D4F009388
:101644005E0410935F04009159040031E0F4BADEA3
:1016540032D011F400271EC0009159040395009361
:101664005904082F192FEA2FFB2F0995002311F095
:1016740001E010C0E5E5F4E001851285005E1F4F2E
:1016840001871287E0CF0027009359049BDE05D021
:10169400CACF02E0E4E00C9467170F5F1F4F2F4F8F
:1016A4003F4F11C004171507260737070895082F61
:1016B400192F2A2F3B2FFDCE0187128723873487CA
:1016C40007C0E5E5F4E000831183228333830895A2
:1016D400058716872787308B08959FDF002339F00D
:1016E4000A9519F00A9519F002C001E0089500273F
:1016F40008950E9456171DD0BDDEE3DF0DD020D023
:101704001DD0002700935904482F592F0A2F1B2F4F
:10171400E4DFE4E00C94671700915404112740912E
:10172400530455270E943816212F210F220B322FE4
:101734000895A02FB12F842F952F0895D6DE05C0CC
:1017440040815181628173810895058316832783C3
:10175400308708952FDEA0DE10F407DE01C046DFD7
:101764003FD039F00A9519F00A9529F004C001E038
:1017740011C000270FC0082F192F2A2F3B2F59DE25
:1017840008DE10F06CDE01C075DE07D000E0A007B3
:10179400B00731F7E8E00C94631793DF0091540429
:1017A400112722273327CCDFA0DECFDF8F3F0FEFB7
:1017B40090070895442D552D0E94561641505040CF
:1017C400042F152F462D572D0C943816442D552DC6
:1017D4000E945616452B082F192F2A2F3B2F0895A8
:1017E400442D552D062D172D18DF0023089504D000
:1017F400B1DFE4E00C9467170E94561762DE009094
:10180400540411242224332480819181A281B38140
:10181400080E191E2A1E3B1E058216822782308658
:101824002227209359040895C5DD36DE10F49DDD8A
:1018340001C0DCDED5DFB9F00A9519F00A9521F074
:1018440003C001E011C00FC0082F192F2A2F3B2F0E
:1018540056DE9FDD10F003DE01C00CDE9EDFA00724
:101864000FE0B00739F70027E8E00C946317C4DFF2
:10187400DBDFE4E00C9467170E945417802F912F4C
:10188400442E552E9DDD17DFF1F00091590410917F
:101894005A04065F1D4F39D0B1F03FD00E94B015F5
:1018A40011272091590430915A04020F131F12502A
:1018B40098F0422F532F84DDB4DD002321F00AE099
:1018C40012E023D011F4002710C012D0132F11708E
:1018D400158378DDE2DE01C00BD0082F192FE42D2B
:1018E400F52D0995002371F201E0E6E00C946517EB
:1018F4008FDE0E94B0151127E5E5F4E024813581DF
:10190400200F311F24833583089500935B041093C3
:101914005C040E94B015002308957ACED2DD2227FC
:101924002093590420935A04A7CF0E94561720915C
:101934004204245039F0225029F0265049F023570C
:1019440049F00AC09ADD11F4D4DE07C050DF05C0A7
:101954008EDF03C0E3DF01C00027E4E00C946717C7
:101964000E94561720914204245039F0225029F045
:10197400265049F0235749F00AC07FDD11F4ADDE4B
:1019840007C0E8DE05C050DF03C076DF01C00027D2
:10199400E4E00C9467170E944E17802F912F842E39
:1019A400952EAC84BD84E02FF12FB0A178D040E215
:1019B40050E0082D192D0E94AD1703E071D040E2CC
:1019C40050E00A2D1B2D0E94AD17BB2309F445C01E
:1019D400BF3008F042C0E82FF92F01A10230E8F12E
:1019E400482E592E01E2400E00E0501E6B2EAA270D
:1019F4004BE33FD031F05FD020F4B02F082F0F5DC0
:101A0400B01BBD3050F54EE234D069F054D058F4D8
:101A1400602E282F2F5D621A0F5F1F4F402E512E0C
:101A2400AB2FA619AA9509E06016B8F4A430A8F45F
:101A340077247A926A928196482F592F082D192D6E
:101A44000E949617BB27BA93AA93442D552D0A2DAD
:101A54001B2D0E94961701E001C00027EEE00C94B4
:101A64005F17E82FF92F21938E2F9F2FE02FF12F4F
:101A7400089550E0082F192F0F5D1F4F0E94BE17C5
:101A8400202F212B0895402F512F622F732F062DC5
:101A9400172D21D0402E512E012B089517D008E088
:101AA40010E01A930A9308950E949617082D192D91
:101AB4002A2D3B2D0895282F392F2F5D3F4F402F7E
:101AC400512F421B530B4B17504008950087118729
:101AD4002287338708953FD0042F152F262F372FC1
:101AE400EADD49F12AE032E000910A0210910B028A
:101AF4000639124029F0E82FF92F06850061068780
:101B0400E22FF32F048115810030114029F4E82FCE
:101B1400F92F068500640BC0E22FF32F0481158191
:101B24000038104029F0E82FF92F06850061068758
:101B340047DCC1DD19F4002711270AC0E82FF92F6B
:101B4400068506FF03C000E011E002C000E810E0D3
:101B54008991999108959A938A93802F912F08954A
:101B64000E944E172397602E712E0FE099DF4427B1
:101B74005527062D172D0E94AD17009142040F37EB
:101B840009F05EC0CADEEFD0012B022B032B09F44F
:101B9400A8C00C2F1D2F1A930A93462D572DBDDE76
:101BA400FADE002309F49DC0E0915B04F0915C042B
:101BB400018D01FD96C0E62DF72D0685046006878C
:101BC40003E06EDF4DE152E00C2F1D2F0E5FDBD0E2
:101BD40069F4A3DEC8D0013012402040304008F040
:101BE40080C008E0E62DF72DB9D024C003E058DF0B
:101BF40040E152E00C2F1D2F0E5FC5D009F071C0DB
:101C04008CDE0E5F1F4F0E94DB153DDF09F469C0B7
:101C1400F2DC452B462B472B41F07FDEA4D001306C
:101C240011402040304008F05CC0E5DCE62DF72D83
:101C34000487158772DE9BD0E62DF72D47DF89C018
:101C4400A7D0828C938C04891589A02EB12E008193
:101C5400053E09F446C00081002309F442C003850F
:101C64000E7DF9F5048D158D268D378D012B022BF4
:101C7400032B09F436C003E013DF4DE152E07ED0BC
:101C8400C9F486D0048D158D268D378D0130124010
:101C94002040304030F508E0E62DF72D0687002778
:101CA40011270487058702E080169106A106B10674
:101CB400F0F546C003E0F4DE40E152E05FD089F481
:101CC40067D0038500FF05C0E62DF72D0685046067
:101CD400068763D018F0EADEC3DB01C0CBDBD3DEBA
:101CE40011F4002737C054D0848D958DA68DB78DFF
:101CF400082F192F2A2F3B2F83DC452B462B472BEC
:101D040039F0813001E0900700E0A007B00710F53A
:101D140080519040A040B040082F192F2A2F3B2F0C
:101D240072DBE62DF72D0487158737D048F00EEFC8
:101D3400800E0FEF901EA01EB01EB8DE92DB01C015
:101D440099DBE62DF72DAADE2FD0062D172D0E9444
:101D5400961701E02396ECE00C945F1706870027A2
:101D6400048705870895065F1F4F0C94DB150E5FEB
:101D74001F4F0E94DB1542E00C94881600915E040C
:101D840010915F04085F1F4F0E941615012B0895E0
:101D9400E0915E04F0915F04089502E0801600E093
:101DA4009006A006B006089540915E0450915F0429
:101DB4000895BEDA41F073DE16D0E6DF11F401E0D7
:101DC40003C00AD0C1F70027E4E00C9467170BD0D6
:101DD4000E947217012B089542EB5DE0082F192F22
:101DE400BFDD002308954A2F5B2F082F192F089574
:101DF4009FDA39F054DEEBDF11F401E003C0ECDFCD
:101E0400C9F70027E4E00C94671792DA39F047DE4B
:101E1400DEDF11F401E003C0DFDFC9F70027E4E0EF
:101E24000C94671785DA61F0E82FF92F0DD0EA2FAB
:101E3400FB2F86DC37DC11F401E003C0CDDFA1F712
:101E44000027E4E00C94671700851185228533850B
:101E540008959A938A932F970027112722273327CF
:101E64002ADC09F476C02AE032E0EAE0F2E0E2504B
:101E7400FE4F0081118105351A4A09F06AC02254C7
:101E84003E4FE22FF32F0081003809F062C0048135
:101E940000934204D9DF0FDC09F45BC08AE092E0CE
:101EA40000914204045029F0025019F0065029F11F
:101EB40050C054D0438554856BD041875287638783
:101EC4007487458756876787708BE82FF92F0681BB
:101ED400178144E00E944F16177F40915404552700
:101EE4000E9456160093530417DCE2E4F4E04185A3
:101EF40052856385748522DC2AC030D0418D528D91
:101F040047D0458356836783708701E00093530469
:101F1400E82FF92F01A112A123A134A102306FDA15
:101F240030F001A112A123A134A19ADA01C0A2DAEE
:101F3400C3DBE0DA088719872A873B8700270C87E9
:101F44000D8746D0202F212B11F00093530401E07C
:101F540001C000272F968991999108950B96E82F37
:101F6400F92F418952896389748903811481222755
:101F74003327400F511F621F721FE2E4F4E04183D4
:101F8400528363837483E82FF92F05811127089501
:101F94000E9438162281209354044189528963890E
:101FA400748903801480400D511D631F731F222701
:101FB400400F511F631F721FE2E4F4E008950C2FD9
:101FC4001D2F085F1F4F1A930A9341E252E00895B0
:101FD4000C2F1D2F085F1F4FAACA9A938A9300E4FF
:101FE40010E020E030E067DB51F18AE092E00AE0A3
:101FF40012E00E94B015013011F505E051DD48E30F
:1020040052E00AE012E00F5FBEDEC9F40FE700936E
:1020140042040AE012E004561F4FA9DEE2E4F4E0B1
:102024004BDB805B9F4F082F192F0E94DB1542E08A
:102034000E948816E6E6FF2788DB01E001C000273E
:102044008991999108959A938A93992781E0883088
:1020540038F4082F0AD00CD00CF493958395F7CF5D
:10206400092F899199910895082DD3C9402F512F93
:10207400E05FFB4F0081003008959A938A93239781
:102084005DD0009142040F3709F547DC6CDE003067
:1020940018402040304091F50C2F1D2F1A930A93BD
:1020A400482F592F3ADC77DC002341F1E0915B049F
:1020B400F0915C04018D01FF21C0E82FF92F068502
:1020C40004604CDE2ADC53DE45D033C061DE028D71
:1020D400138D44895589242F352F4081453E71F055
:1020E4004081442359F0438544FF08C0448D558DF5
:1020F400668D778D452B462B472B11F000271AC090
:1021040044275527E82FF92F4487458702301407C1
:102114002407340728F072D940915404A5D901C08A
:10212400A9D9E82FF92FBADC3FDE082F192F0E9416
:10213400961701E02396899199910895802F912F04
:102144000FE010E01A930A9344275527082F192FFC
:102154000C94AD17E82FF92FB9CCFDDC4FE350E117
:10216400E4DB002331F0E82FF92F068502600687AF
:1021740003C00FE095DC04D001E0899199910895A2
:10218400E3CFE9DC4FE350E1EBDB002331F0E82F50
:10219400F92F068502600687EFCF0FE081DCF0DFC0
:1021A400EBCFE02FF12F268521FF06C04DDEE2E4C0
:1021B400F4E08EDA01E00895002708959A938A9353
:1021C400BDDFE2E4F4E00585168527853089418585
:1021D40052856385748566DA62DC19F446E252E05E
:1021E40002C04FE252E0082F192F0E944815E2E482
:1021F400F4E00585168527853089ACDF0685026005
:102204000687BACF0FE414E00C941616A4DCF1D8B8
:1022140021F211D069F043DC44E152E0082F192F78
:10222400B3DD31F0E82FF92F068500680687A4CFC7
:10223400D3DD79F7B2CF082F192F085F1F4F77D955
:10224400012B089588DCC8DD09F4A7CFF4DFD9F3A6
:1022540026DC44E152E0082F192F96DDA1F3E82F84
:10226400F92F06850068068787CF97CF0E945617F7
:10227400802FA42FB52F0FE013DC442755270A2FF6
:102284001B2F0E94AD178823C1F08830B0F4009151
:102294001004083091F4082FE8DEE8DE64F4465FA9
:1022A4005B4F0A2F1B2FBEDD002329F0EA2FFB2FE3
:1022B40006850068068701E001C00027E4E00C946D
:1022C40067170E9451172F97802E442E552E0023F6
:1022D40009F47BC008E0801608F077C00091100470
:1022E400083009F072C0485F5F4F0C2F1D2F9ADD34
:1022F400002309F46AC0E5E5F4E080819181A281BC
:10230400B38166DE012B09F460C0009142040F37EB
:1023140009F459C0CCD909F458C0E42DF52D06852B
:1023240037DD02FF03C00385016002C003850E7F11
:102334000387082F192F53D009F447C0082D4AD01A
:10234400202F312F065F1B4FEC2FFD2F389647E0CF
:1023540050E00E942717E22FF32FE05FFB4F00812C
:1023640000680083E42DF52D0685205F3B4FE22FA6
:10237400F32F02FF03C00081046002C000810B7FC1
:102384000083A1E0A830F8F40A2F24D0802F912FE5
:10239400865F9B4FE82FF92F4080518062807380C5
:1023A40063DEE65FFB4F0ED84016510662067306E5
:1023B40041F4A81531F0082F192F47E050E00E948E
:1023C4002717A395DFCF01E001C000272F96E9E08E
:1023D4000C946217112747E050E00C9438162A2F0A
:1023E4003B2F24D8002308959A938A93202F002307
:1023F400A9F0283098F400911004083079F407E02B
:102404004FDB5527022F47E00E943816065F1B4F0B
:1024140040E050E00E94AD1701E001C0002789911F
:1024240099910895002321F0083010F401E00895F3
:1024340000270895002369F0083058F416DE18DEEA
:1024440044F406FF03C000E011E0089500E810E042
:102454000895002711270895002379F0083068F4BF
:1024640004DEE05FFB4F208120303CF4025F1B4F11
:10247400E02FF12F0081118108950027112708957D
:102484000E9452172F97009142040F3709F45CC041
:10249400DADD11274DE050E00E943816802F912F8D
:1024A40044E152E00C2F1D2F84DC002309F44CC0BE
:1024B400AA276EDC848F958FA68FA78F0E94E209CE
:1024C40090DF09F441C0488459846A847B84882756
:1024D4009927A1E0A830B0F50A2FC7DDC7DD84F540
:1024E400465F5B4F0C2F1D2F9DDC002349F1042D0B
:1024F400152D262D372DDFD839F104E42AD00A2FE3
:10250400005D27D00DE325D0CADA4C2F5D2F4E5F36
:102514005F4F082F192F065F1D4F0E9496170896CC
:102524000DE017D00AE015D00027E82FF92FE65F59
:10253400FD4F0083042D152D262D372D52DF21F05C
:10254400A395C8CF01E001C000272F96E8E00C94C2
:102554006317E82FF92F0196E65FFD4F0083089576
:10256400E6E6FF274AE050E00C942717F4DA0091DE
:102574004204E82FF12F008300915404018363DDAA
:10258400E82FF92F028300E3038389919991089539
:102594000E9454172F97CDD8442E552E01E480DA8B
:1025A400EFDD4A2F5B2F0C2F1D2F22DC002309F4B3
:1025B4005AC0EEDB06810E37D9F50E2F1F2FAA273E
:1025C400209159042A952093590491F10052104006
:1025D40001C02EC0E02FF12F23852F3049F5A35FD2
:1025E400A23430F521813DDA23813BDA258139DAC1
:1025F400278137DA218535DA268533DA208931DAFD
:1026040022892FDA24892DDA26892BDA208D29DAFA
:10261400248D27DA268DE82FF92F21938E2F9F2FD3
:1026240022272083E02FF12F2081203448F219C083
:1026340036DABADB042D152D0E9496170EE2E42D2E
:10264400F52D008703E02CDAAFDB485F5F4F042DE4
:10265400152D075F1F4F0E9496170027E42DF52DB7
:10266400048701E001C000272F96E6E00C9465176B
:102674000E944C17802EA42EB52ECE84DF84002316
:1026840009F467C008E0801608F063C0EDDCE05F81
:10269400FB4F808180300CF05CC0E6DCE25FFB4FD6
:1026A400008111810A151B0508F453C00A2D0B295A
:1026B40009F44FC086FF04C0662401E0702E03C0F5
:1026C40000E8602E772449D00A2D1B2D0E94A10911
:1026D4000A2D1B2D7BD879F00E945D0BD1F10A2DB8
:1026E4001B2D68D8005F1F4F7A926A92065F1D4FB8
:1026F400402F512F28C00E945D0B59F100E112E0D8
:1027040006191709262D372D205130403A932A9364
:10271400065F1D4F402F512F0C2D1D2D0E94961723
:102724008F5F9F4FAF4FBF4F0E94590B91F0062D03
:10273400172D0051104020E130E03A932A934AE0EB
:1027440052E0C00ED11E0C2D1D2D0E94961701E0E3
:1027540001C00027E0E10C945D1700E012E0462D73
:10276400572D0E945616402E512E08950E944A1746
:10277400802EC42ED52EE888F988009142040F37A4
:1027840009F473C0882009F470C008E0801608F0CA
:102794006CC06ADCE05FFB4F808180300CF065C068
:1027A40082FD63C061DCE25FFB4F008111810C1587
:1027B4001D0508F45AC00C2D0D2909F456C086FFD6
:1027C40004C0662401E0702E03C000E8602E772464
:1027D400C4DF0C2D1D2D0E94A109882E992EAA2E2E
:1027E400BB2E0C2D1D2D0E94E80BA1F00E945D0B49
:1027F400E1F10C2D1D2D0E94DC0B802F912F4096B2
:102804007A926A9236D00E949617082D192DE7DD28
:1028140061F129C00E945D0B41F180E192E08619CB
:102824009709062D172D005110401A930A9321D0B1
:102834003BD9D7DDD1F00FEF801A900AA00AB00A75
:10284400862D972D8051904031D90E945D0B69F0FF
:1028540000E126D9E80EF91E4E2D5F2D0AE012E0A4
:1028640023D9BFDD11F001E001C00027E2E10C949F
:102874005B174E2D5F2D865F9D4F082F192F0895EE
:102884000E9455172A97A02FB12F44E152E091DA04
:10289400002309F47CC0EA2FFB2F04851585012B46
:1028A40009F075C008E3FCD87ED00AE014E074D0C7
:1028B400EAE0F4E00E94E4090E945D0B09F467C0B9
:1028C4007EDB0AE012E00E946E15802F912F012B0F
:1028D40009F45DC0E82FF92F0081043409F044C0E5
:1028E40002810D3309F040C0418000ED400EE1F15A
:1028F40008E04016C8F5082F192F0D5F1F4F0E94DE
:10290400CB170930104080F5CAD840E250E00C2FB4
:102914001D2F0E5F1F4F0E94AD17082F192F0D5F3B
:102924001F4F0E94CB171A930A930396482F592FCF
:102934000C2F1D2F0E5F1F4F0E9496174C2F5D2FDB
:102944000A2F1B2F62DA002379F00A2F1B2F42DB98
:10295400012B29F0EA2FFB2F068500680687042D3A
:1029640039DD065F1B4F18D0EAE0F4E00E94E40969
:102974000E945D0B61F023DB002711270E946E1576
:10298400802F912F012B09F0A5CF01E001C0002772
:102994002A96E5E00C946617EA2FFB2F389647E059
:1029A40050E00C942717442755270AE014E00C94B0
:1029B400AD172F9703E174D84427552702E414E098
:1029C4000E94AD1708E36CD8EEDF06E611270E94DB
:1029D4003407002331F10A9519F00A9529F021C032
:1029E40038DA002321F41DC0F8DA0023D1F00FE413
:1029F40014E00E94E215002329F00C2F1D2F40DF64
:102A0400002369F40BE414E00E9416160E943C0AA9
:102A14000E946A0B0C2F1D2F33DF002311F001E0FD
:082A240001C000272F96089560
:04023E00FFFFFFFFC0
:100210004154520053494F32494445200043464718
:100220000020090D0A00433A28524F4F5429002854
:0E0230005355424449522900434430303100B6
:102A2C0028813981622F732F21503040672BD9F0C8
:102A3C00E02FF12F6081E42FF52FC895601571F010
:102A4C00E02FF12F0081E42FF52FC895001618F414
:102A5C0001E010E00AC00FEF1FEF07C00F5F1F4F20
:102A6C004F5F5F4FDFCF002711272296089505D0C7
:102A7C000F5F1F4F008311830895E82FF92F0081FA
:102A8C00118108959A938A938A819B81282F392FDB
:102A9C000197232B59F0E42FF52F4F5F5F4FC8950B
:102AAC00E02FF12F01920E2F1F2FF0CF89919991CA
:102ABC0022960895E02FF12FC895002031F0C8958B
:102ACC00041629F00F5F1F4FF5CF0027112708952B
:102ADC000E945417442E552E8E819F81202F212B1E
:102AEC0021F0E82FF92F00831183C7DF012B41F070
:102AFC002BD021F020D011F0BADFFACF25D019F469
:102B0C000027112715C0E82FF92FA081B1811CD007
:102B1C0069F011D011F4ABDFFACF0027E82FF92FB1
:102B2C0020813181E22FF32F0083A1DF0A2F1B2F8D
:102B3C00E8E00C946517A1DFE02FF12F4081042D04
:102B4C00152DB8DF012B089598DFE02FF12F0081B0
:042B5C0000230895B5
:102B6000E02FF12F00810895E02FF12F0081112730
:102B70000895E02FF12F008111810895E02FF12FAA
:102B800020810181122F0895F4CFF3CF402F512FD0
:102B9000E02FF12F0081302F22271127E42FF52F6E
:102BA0000180322E202D33290280312E102D332921
:102BB0004381042F0895E02FF12F0081118122819C
:042BC00033810895C0
:102BC400E02FF12FE199FECF19D0E09A0DB30A3A24
:102BD40091F4E199FECF05E61BD0E199FECF06E61C
:102BE40017D0E199FECF07E613D0E199FECF08E6AE
:102BF4000FD001E0089500270895F89404E610E04A
:102C04001FBB0EBB089510E01FBB0EBB019107C094
:102C140010E01FBB0EBBE09A0DB3019308950DBBEA
:102C2400E29AE19A78940895E02FF12FE199FECF8A
:102C3400E4DF0FEFF4DFE199FECFF89405E6E3DF7C
:102C4400E199FECFF89406E6DEDFE199FECFF89431
:102C540007E6D9DFE199FECFF89408E6D4DFE199DD
:0C2C6400FECFCBDF0AEADBDF01E00895C1
:102C7000002411240030010741F01695079510F447
:102C8000040E151E440F551FF5CF002D112D08956C
:0E2C90004A9522F0000F111F0C94481608956B
:0E2C9E004A9522F0169507950C944F1608954E
:102CAC0000241124E0E1EA9552F0001F111F001CD2
:102CBC00111C04161506B8F3041A150AF4CF001FDC
:0C2CCC00111F402D512D0095109508950A
:102CD8000024112422243324E02FE12BE22BE32BC0
:102CE80071F0369527951795079520F4040E151E53
:102CF800261E371E440F551F661F771FEDCF002D68
:082D0800112D222D332D089539
:102D10004A9532F0000F111F221F331F0C948816A2
:022D2000089514
:102D22004A9532F036952795179507950C9491168A
:022D3200089502
:102D34000024112422243324E0E2EA9592F0001FB7
:102D4400111F221F331F001C111C221C331C0416CC
:102D540015062606370688F3041A150A260A370AC2
:102D6400ECCF001F111F221F331F402D512D622D48
:0C2D7400732D0095109520953095089562
:102D8000C895702D3196C895602D3196C895502DF7
:102D90003196C895402D3196C8953196102C01FA80
:102DA000C8953196202CC8953196302C0895F1DFC6
:102DB000041B10E003C0EADF041B150B20E030E029
:102DC00005C0DEDF041B150B260B370BC8F010FC0B
:102DD0001AC03AD0402D38D00417100588F446F4B4
:102DE000E00FF11FC895E22DF32DE019F040099492
:102DF000000F111FE00FF11F27D0202C25D0302C01
:102E0000E22DF32D099411F4BEF7ECCF31960EF0BC
:102E1000319650E060E070E017D0402D4B3F68F0F5
:102E200079F34F3F41F04E3F21F00ED0702D0CD082
:102E3000602D0AD0502D08D0402D041B150B260BF9
:0E2E4000370B11F3E8F2E2CFC89531960895F2
:102E4E00BF93AF93A02FB12F02C001900D924150AE
:0A2E5E005040D8F7AF91BF910895DE
:102E6800BF93AF93A02FB12F03C0C89531960D9291
:0C2E780041505040D0F7AF91BF91089539
:0E2E8400002401C0019201501040E0F70895B3
:022E920000003E
:102E9400FA92EA92DA92CA92BA92AA929A928A928E
:102EA4007A926A925A924A92BA93AA939A938A937A
:022EB40008957F
:102EB600FF84EE84DD84CC84BB84AA8499848884D0
:102EC6007F806E805D804C80BB81AA8199818881DC
:0E2ED600F0E00FB6F894CE0FDF1F0FBE089588
:102EE40028813981622F632B79F0E02FF12F6081E3
:102EF400E42FF52F7081671739F40F5F1F4F4F5F71
:102F04005F4F21503040EECF232B51F0E02FF12FB3
:102F140000811127E42FF52F2081021B104002C0ED
:082F24000027112722960895F1
:102F2C0068817981202F312F062E172E6150704029
:102F3C00012859F0E42FF52F0080E22FF32F019296
:0E2F4C002E2F3F2F4F5F5F4FEFCF229608953D
:102F5A009A938A938A819B81E02FF12F282F392F08
:102F6A000197232B11F04193F9CF899199912296D8
:022F7A000895B8
:102F7C00E02FF12F3081341739F021910E2F1F2FB4
:0A2F8C002223B1F700271127089552
:102F9600E02FF12F2081222311F03196FBCFE01B89
:082FA600F10B0E2F1F2F0895FF
:00000001FF
